S0220000687474703A2F2F737265636F72642E736F75726365666F7267652E6E65742F1D
S12300000C9438000C9475150C94F71B0C945F000C945F000C945F000C945F000C945F002D
S12300200C945F000C94B31C0C945F000C9493200C945F000C944E160C9428160C94161550
S12300400C9474210C945F000C94E9200C945F000C9420220C94E8210C945F000C945F0037
S12300600C945F000C945F000C945F000C945F0011241FBECFEFD0E1DEBFCDBF14BEA895C7
S123008088E10FB6F89480936000109260000FBE15E0A0E0B1E0EAEBF7E402C005900D92B4
S12300A0AA31B107D9F716E0AAE1B5E001C01D92A03BB107E1F70E947A0D0C94DC230C9480
S12300C0000020E030E0D901AC54BF4F0E94BE23802DF901E05CFE4F80832F5F3F4F203AF8
S12300E0310589F720E030E0D901A857BE4F0E94BE23802DF901E75CFE4F80832F5F3F4F77
S12301002530310589F712BC11BC089520E030E0F901E05CFE4F8081D901AC54BF4F082EE6
S12301200E94CB232F5F3F4F203A310589F712BC11BC08954E9B11C020E030E0D90150963D
S12301400E94BE23802DF901E052FE4F80832F5F3F4F203A310591F0F1CF20E030E0D90118
S1230160A859BD4F0E94BE23802DF901E052FE4F80832F5F3F4F203A310589F712BC11BCFB
S123018008954E9B11C020E030E0F901E052FE4F8081D9015096082E0E94CB232F5F3F4FD8
S12301A0203A310591F0F1CF20E030E0F901E052FE4F8081D901A859BD4F082E0E94CB2333
S12301C02F5F3F4F203A310589F712BC11BC089520E931E0D9010E94BE23802D20553140AD
S12301E0F901E058FD4F80832F5A3E4F81E0203F380781F712BC11BC089520E430E0F901A7
S1230200E058FD4F8081D901A05BBE4F082E0E94CB232F5F3F4F203A310589F712BC11BCE6
S12302200895A2E0B0E00E94BE23802D90E090931F0180931E0120911E0130911F01A3E0C2
S1230240B0E00E94BE23802D90E0982F8827820F931F90931F0180931E01A4E0B0E00E9486
S1230260BE23802D90E090932101809320012091200130912101A5E0B0E00E94BE23802D09
S123028090E0982F8827820F931F9093210180932001A6E0B0E00E94BE23802D90E09093DF
S12302A00101809300012091000130910101A7E0B0E00E94BE23802D90E0982F8827820FF1
S12302C0931F9093010180930001A1E0B0E00E94BE23802D80931A05A8E0B0E00E94BE2321
S12302E0802D80931301A9E5B1E00E94BE23802D80932A01A2E0B4E00E94BE23902D892F8B
S12303008150843078F080912A01843039F481E08093180183E68093C00506C082E08093C6
S1230320180102C090931801A9E0B0E00E94BE23802D80931201AEE0B0E00E94BE23802DE5
S123034080932301ABE0B0E00E94BE23802D80931B01ACE0B0E00E94BE23802D80931C016C
S1230360AFE6B1E00E94BE23802D80931D01A2EFB1E00E94BE23802D809389058091890560
S1230380882319F081E080938905ADE0B0E00E94BE23802D26E0829FC00111249093150100
S12303A080931401A1E7B1E00E94BE23802D8093E405A0E7B1E00E94BE23802D8093E2058A
S12303C08AE08093110681E080930F06AFE8B1E00E94BE23802D80932B01A4EFB1E00E949F
S12303E0BE23802D24E1829FC00111249093BB058093BA05A5EFB1E00E94BE23802D809332
S1230400B705A6EFB1E00E94BE23802D8093B505A7EFB1E00E94BE23802D8093B405A8EF3F
S1230420B1E00E94BE23802D90E09093B3058093B2052091B2053091B305A9EFB1E00E9436
S1230440BE23802D90E0982F8827820F931F9093B3058093B205ABEFB1E00E94BE23802DE1
S123046090E090932D0180932C0120912C0130912D01ACEFB1E00E94BE23802D90E0982F17
S12304808827820F931F90932D0180932C01ADEFB1E00E94BE23802D90E090932F018093A2
S12304A02E0120912E0130912F01AEEFB1E00E94BE23802D90E0982F8827820F931F90938E
S12304C02F0180932E01AFEFB1E00E94BE23802D90E090933101809330012091300130919B
S12304E03101A0E0B2E00E94BE23802D90E0982F8827820F931F909331018093300120E0C2
S123050030E0D901A25ABE4F0E94BE23802DF901E05EFC4F8083D901AE58BE4F0E94BE23BE
S1230520802DF901EF53FA4F8083D901A458BE4F0E94BE23802D808B2F5F3F4F2A303105B8
S123054001F7A7E0B2E00E94BE23802D80933401A3E0B2E00E94BE23802D8093350120E080
S123056030E0F901E251FA4F84E6808BD901A45EBD4F0E94BE23802D80832F5F3F4F2031F4
S1230580310579F720E030E0D901A759BE4F0E94BE23802DF901EB5DFE4F80832F5F3F4FDC
S12305A02430310589F720E030E0D901A25DBD4F0E94BE23802DF901E051FB4F80832F5F02
S12305C03F4F2031310589F7ADE6B1E00E94BE23802D80932201A1EFB1E00E94BE23802DA7
S12305E080938805A0EFB1E00E94BE23802D80932901A6E0B2E00E94BE23802D809324014A
S123060020E030E0D901AA54BC4F0E94BE23802DF901E65DFC4F80832F5F3F4F2031310585
S123062089F7A7ECB3E00E94BE23802D80933701A8ECB3E00E94BE23802D80933801A8EE5C
S1230640B3E00E94BE23802D90E090931A01809319012091190130911A01A9EEB3E00E9485
S1230660BE23802D90E0982F8827820F931F90931A0180931901AAEEB3E00E94BE23802DF9
S12306808093760512BC11BC089580911E0190911F01A2E0B0E0082E0E94CB2380911E0117
S12306A090911F01892F9927A3E0B0E0082E0E94CB238091200190912101A4E0B0E0082EE5
S12306C00E94CB238091200190912101892F9927A5E0B0E0082E0E94CB238091000190918B
S12306E00101A6E0B0E0082E0E94CB238091000190910101892F9927A7E0B0E0082E0E947C
S1230700CB2380911301A8E0B0E0082E0E94CB2380911201A9E0B0E0082E0E94CB2312BC13
S123072011BC089580E0A1EFB1E0082E0E94CB238AE0A0EFB1E0082E0E94CB238091890515
S1230740A2EFB1E0082E0E94CB2384E0A9E5B1E0082E0E94CB2385E0ACE0B0E0082E0E940B
S1230760CB2382E3AFE6B1E0082E0E94CB2324E1A1E7B1E0022E0E94CB2391E0A0E7B1E0CF
S1230780092E0E94CB2388ECA4EFB1E0082E0E94CB23A5EFB1E0092E0E94CB23A6EFB1E01E
S12307A0022E0E94CB238AE5A7EFB1E0082E0E94CB2388EEA8EFB1E0082E0E94CB2383E052
S12307C0A9EFB1E0082E0E94CB2380912C0190912D01ABEFB1E0082E0E94CB2380912C016A
S12307E090912D01892F9927ACEFB1E0082E0E94CB2380912E0190912F01ADEFB1E0082E48
S12308000E94CB2380912E0190912F01892F9927AEEFB1E0082E0E94CB23809130019091E4
S12308203101AFEFB1E0082E0E94CB238091300190913101892F9927A0E0B2E0082E0E9496
S1230840CB238CEDA7E0B2E0082E0E94CB2386EEA3E0B2E0082E0E94CB232CE132E088EC6C
S1230860D901082E0E94CB232F5F3F4F82E02C323807A9F782E2AFE8B1E0082E0E94CB23C7
S123088081E0A6E0B2E0082E0E94CB2312BC11BC0895CF92DF92EF92FF920F931F93CF9343
S12308A0DF93C0E0D0E0A5E0B2E00E94BE23202D30E040E050E0A3EDB3E00E94BE23602DF8
S12308C06E01CC0CDD1C8AE393E0C80ED91EF601E080F18070E080E090E00E942F2300E06B
S12308E010E0A80197010E942F2324E630E040E050E00E94812379018A01CA01B90124EF82
S123090031E040E050E00E942F2328EC30E040E050E0E20EF31E041F151FA80197010E94CF
S12309208123CA01B9012FEF30E040E050E00E942F2325E030E040E050E00E94812382E00B
S1230940220F331F441F551F8A95D1F7CA01B90124E630E040E050E00E948123F601318372
S123096020832196C732D10509F09DCFC0E0D0E0A9ECB3E00E94BE23202D30E040E050E03D
S1230980A3EDB3E00E94BE23602D6E01CC0CDD1C88E893E0C80ED91EF601E080F18070E018
S12309A080E090E00E942F2300E010E0A80197010E942F2324E630E040E050E00E948123BA
S12309C079018A01CA01B90124EF31E040E050E00E942F2328EC30E040E050E0E20EF31EAC
S12309E0041F151FA80197010E948123CA01B9012FEF30E040E050E00E942F2325E030E009
S1230A0040E050E00E94812312E0220F331F441F551F1A95D1F7CA01B90124E630E040E0BA
S1230A2050E00E948123F601318320832196C732D10509F09DCFC0E0D0E0AAECB3E00E94E8
S1230A40BE23202D30E040E050E0A3EDB3E00E94BE23602D6E01CC0CDD1C86ED93E0C80ED5
S1230A60D91EF601E080F18070E080E090E00E942F2300E010E0A80197010E942F2324E690
S1230A8030E040E050E00E94812379018A01CA01B90124EF31E040E050E00E942F2328ECA6
S1230AA030E040E050E0E20EF31E041F151FA80197010E948123CA01B9012FEF30E040E020
S1230AC050E00E942F2325E030E040E050E00E948123A2E0220F331F441F551FAA95D1F760
S1230AE0CA01B90124E630E040E050E00E948123F601318320832196C732D10509F09DCF84
S1230B00C0E0D0E0A4E0B2E00E94BE23202D30E040E050E0A3EDB3E00E94BE23602D6E0199
S1230B20CC0CDD1C84E294E0C80ED91EF601E080F18070E080E090E00E942F2300E010E08D
S1230B40A80197010E942F2324E630E040E050E00E94812379018A01CA01B90124EF31E0FE
S1230B6040E050E00E942F2328EC30E040E050E0E20EF31E041F151FA80197010E948123DA
S1230B80CA01B9012FEF30E040E050E00E942F2325E030E040E050E00E948123E2E0220FBC
S1230BA0331F441F551FEA95D1F7CA01B90124E630E040E050E00E948123F601318320833E
S1230BC02196C732D10509F09DCFDF91CF911F910F91FF90EF90DF90CF900895EAE7F0E0EC
S1230BE0108280E280937C0080E880BF87EE808311B808950F931F93CF93DF93282F30E05A
S1230C00F901EE0FFF1FEE5FFE4F0081118143E0033F140718F0E2E3F0E04CC053E00F3D66
S1230C20150718F0EAE0F0E045C0C0E0D0E087E290E0A901489F9001499F300D589F300D49
S1230C401124D901AC0FBD1FAA0FBB1FA65CBC4F8D919C9111978017910730F5FE0131973C
S1230C60E20FF31FEE0FFF1FE65CFC4F20813181608171814D915C91FE01EE0FFF1FEE0FBD
S1230C80FF1FEC0FFD1F3596201B310BC901880F991F880F991F641B750B820F931F0E948D
S1230CA05A23E60FF71F06C02196C732D10549F6E8ECF0E0CF01DF91CF911F910F910895EC
S1230CC00F931F93CF93DF93AC01E0E0F0E0EF01CC0FDD1FDE01AE58BB4F8D919C91119702
S1230CE048175907C0F56D917C913197EE0FFF1FDF01AE58BB4F8D919C911197681B790BA4
S1230D008D919C91C657DB4F28813981E657FB4F00811181481B590B84E690E0DC014A9FD9
S1230D20C0014B9F900D5A9F900D11240E945A23201B310B0190F081E02D629FC001639F33
S1230D40900D729F900D112464E670E00E945A236E0F7F1F09C03196EA30F10509F0B7CF1C
S1230D6060919E0470919F04CB01DF91CF911F910F9108950F931F93CF93DF93AC018091C9
S1230D80B2049091B3044817590718F4E0EFF0E057C08091CE049091CF048417950718F426
S1230DA0E0E0F0E04DC0E1E0F0E0EF01CC0FDD1FDE01AE54BB4F8D919C911197481759079D
S1230DC0C0F56D917C913197EE0FFF1FDF01AE54BB4F8D919C911197681B790B8D919C913B
S1230DE0E053FB4F20813181C053DB4F08811981481B590B84E690E0DC014A9FC0014B9FAD
S1230E00900D5A9F900D11240E945A23201B310B0190F081E02D629FC001639F900D729F4F
S1230E20900D112464E670E00E945A23E61BF70B07C03196EE30F10509F0B7CFEEEFF0E052
S1230E40CF01DF91CF911F910F910895A89582E50E94752283E10E94752280917C059091D4
S1230E607D05892F99270E94752280917C0590917D050E94752280913205909133050E948A
S1230E80752280912C0590912D050E94752280911C0590911D050E94752280912A059091DA
S1230EA02B050E94752280912805909129050E94752280912405909125050E947522809130
S1230EC08205909183056091180170E00E945A23CB010E947522809181050E94752280917F
S1230EE080050E9475222091EC053091ED058091BC059091BD05E3E096958795EA95E1F7C5
S1230F008170232F3327822B0E9475228091EC059091ED050E9475228091E1050E947522CC
S1230F2080910E060E94752280912205909123050E9475228091BE059091BF059695879595
S1230F400E94752289B186958695817090E0909339058093380583B18695817090E09093FF
S1230F603B0580933A052091930530E0220F331FF901E45DFA4F80819181892F990F990B64
S1230F8093E0220F331F9A95E1F7822B0E947522E0919305F0E0EE0FFF1FE45DFA4F8081EB
S1230FA091810E9475228DEA0E947522809193058F5F80939305883010F010929305089561
S1230FC0CF92DF92EF92FF920F931F93CF93DF93A89588E10FB6F894809360001092600095
S1230FE00FBE0E94C122882309F47AC50E94522290939205809391058236910509F4E8C246
S12310008336910508F041C08035910509F45AC381359105E8F48534910509F4D1C0863460
S1231020910568F48932910509F4ADC48134910509F48DC08832910509F050C581C4863409
S1231040910509F446C18D34910509F047C5BDC18535910509F4FAC38635910548F48235CA
S1231060910509F4ABC38335910509F037C5DDC48835910509F432C48136910509F442C0F5
S12310808735910509F02AC594C38936910509F4CAC28A369105C8F48536910509F408C2B3
S12310A08636910548F48336910509F494C28436910509F013C514C58636910509F4E7C00C
S12310C08736910509F00AC5D5C28037910509F4FEC28137910548F48D36910509F434C17B
S12310E08F36910509F0FAC411C48937910509F46DC48A37910509F471C28837910509F0AC
S1231100EDC46CC281E60E94752280EA0E94752210929205109291050EC0E05CFE4F8081E0
S12311200E947522809191059091920501969093920580939105E0919105F0919205E03AE0
S1231140F10558F382E30E94C6218EE9C7C41092920510929105C0E0D0E00E94C122882369
S123116041F1C0919105D0919205C03AD10589F40E94522290939205809391058E3B910535
S123118019F4C6E1DAEF15C0809191050E947522FBCF0E945222C05CDE4F8883809191053E
S12311A09091920501969093920580939105C0E0D0E021964AEFC030D40708F091C4CDCF85
S12311C0C0E0D0E00E94C122882309F459C00E9452228A3B910509F083C488E10FB6F8940A
S12311E080936000109260000FBE10929205109291053EC0885B0E9475228DEF0E94752269
S123120020919105309192058AEF90E0289FE001299FD00D389FD00D112407C0DE010E94C4
S1231220BE23802D0E947522219620919105309192052F5F3F4F8AEF90E0AC01249FC00157
S1231240259F900D349F900D112421503040C817D90720F3822F885B80950E9475228091DE
S12312609105909192050196909392058093910580919105909192058430910508F4BACFF4
S123128021965AEFC030D50708F02AC49BCF86E60E94752280EA0E9475221092920510920B
S12312A091050EC0E052FE4F80810E947522809191059091920501969093920580939105B4
S12312C0E0919105F0919205E03AF10558F389E905C4109292051092910500E010E00E9472
S12312E0C122882349F1C0919105D0919205C03AD10591F40E945222909392058093910575
S1231300893B910519F406E11AEF16C0E0918F05F0919005099510C00E945222C052DE4FBE
S1231320888380919105909192050196909392058093910500E010E00F5F1F4F8AEF0030F0
S1231340180708F0CDC3CBCF8DE60E94752289E00E94752280911E0190911F010E94752250
S123136080911E0190911F01892F99270E94752280912001909121010E9475228091200167
S123138090912101892F99270E94752280910001909101010E9475228091000190910101B2
S12313A0892F99270E947522809113010E947522809112010E947522AAE0B0E00E94BE2320
S12313C0802D0E94752282E989C31092920510929105C0E0D0E00E94C1228A3008F461C04F
S12313E00E94522290931F0180931E0100911E0110911F010E945222982F8827800F911F22
S123140090931F0180931E010E945222909321018093200100912001109121010E94522239
S1231420982F8827800F911F90932101809320010E94522290930101809300010091000199
S1231440109101010E945222982F8827800F911F90930101809300010E94522280931301A4
S12314600E945222809312010E945222AAE0B0E0082E0E94CB230E94681C0E945222823B3D
S1231480910551F40E944503E0918F05F09190050995CFE6DAEF05C0E0918F05F09190056C
S12314A0099521964AEFC030D40708F019C393CF85E60E94752283E10E947522109292051F
S12314C0109291050EC0E05EFC4F80810E947522809191059091920501969093920580937C
S12314E09105E0919105F0919205EA30F10558F380911B010E94752280911C010E9475220B
S123150083E00E94C721809125010E947522809126010E947522809127010E947522809176
S123152028010E947522809114019091150166E070E00E945A23CB010E94752280912201FA
S12315400E947522AEE6B1E00E94BE23802D0E9475228AE90E9475228CE60E94752284E104
S12315600E94752210929205109291050EC0EF53FA4F80810E9475228091910590919205CB
S123158001969093920580939105E0919105F0919205EA30F10558F3109292051092910562
S12315A00EC0EF53FA4F80890E947522809191059091920501969093920580939105E091C2
S12315C09105F0919205EA30F10558F383E986C20E94860085C20E94C10082C20E94260765
S12315E07FC20E945222C82FD0E00E945222C817D90709F075C20E9452228C019093920587
S1231600809391050E9452220817190709F068C20E9452228639910509F062C28091910576
S1231620C05CDE4F4DC00E94C1228530D0F6FBCF0E945222C82FD0E00E945222C817D907F4
S123164009F04EC20E9452228C0190939205809391050E9452220817190709F041C20E9484
S123166052228839910509F03BC280919105C052DE4F26C00E94C1228530D0F6FBCF0E946D
S12316805222C82FD0E00E945222C817D90709F027C20E9452228C0190939205809391056E
S12316A00E9452220817190709F01AC20E9452228F3A910509F014C280919105C058DD4FCD
S12316C088830EC20E94C1228530C8F6FBCFC0E0D0E00E94C122823080F10E9452220E94B9
S12316E052228F38910509F0FBC110929205109291051CC0E058FD4F108180E70E9475225E
S123170082E00E947522809191050E947522812F0E9475228FE80E947522809191059091E9
S1231720920501969093920580939105E0919105F0919205E03AF105E8F221965AEFC0301B
S1231740D50709F4CDC1C5CF0E9452228C010E945222D82FCC27C00FD11F0E9452228C0175
S123176090939205809391050E9452220817190709F0B6C10E945222883A9105A9F4DE0153
S12317800E94C623E0708091910590919205E82BF92BF0939205E0939105DE010F010E9420
S12317A0D72312BC11BC9CC1E0918F05F091900509950E94C122853038F6FBCFCC24DD2457
S12317C00E94C1228330C0F10E9452228C010E945222EC010E9452228D3A910509F080C1C9
S12317E0FC2EEE24E00EF11ED7010E94BE23802D90E0D70111960E94BE23002D10E0102FD6
S12318000027080F191F84E50E94752284E00E947522802F0E9475228E2D0E947522EF2C18
S1231820FF248E2D0E947522012F1127802F0E9475228BEA0E9475220894C11CD11C80E0C9
S1231840C8168AEFD80609F44BC1BACFCC24DD240E94C1228330C0F10E9452228C010E949E
S12318605222EC010E9452228A3A910509F038C1FC2EEE24E00EF11ED7010E94BE23802D60
S123188090E0D70111960E94BE23002D10E0102F0027080F191F85E50E94752284E00E9457
S12318A07522802F0E947522012F1127802F0E9475228E2D0E947522EF2CFF248E2D0E94C6
S12318C075228AEA0E9475220894C11CD11C40E0C4164AEFD40609F403C1BACFC0E0D0E0B3
S12318E00E94C122882359F00E945222873A910509F0F6C0E0918F05F091900509952196DF
S12319005AEFC030D50709F4EBC0EACFC0E0D0E00E94C122882369F00E945222803991050F
S123192009F0DEC00E94FD00E0918F05F0919005099521968AEFC030D80709F4D1C0E8CF70
S1231940C0E0D0E00E94C1228823B1F00E945222873D910509F0C4C08091280590912905E8
S1231960ADE6B1E0082E0E94CB2312BC11BCE0918F05F0919005099521964AEFC030D4076A
S123198009F4AEC0DFCFC0E0D0E00E94C1228823B1F00E945222863D910509F0A1C080912F
S12319A0280590912905AEE6B1E0082E0E94CB2312BC11BCE0918F05F091900509952196B1
S12319C05AEFC030D50709F48BC0DFCFC0E0D0E00E94C122823010F10E945222892B09F0AD
S12319E07FC00E94522286389105C1F489E70E94752285E00E9475228FEC0E9475228FE318
S1231A000E9475228DE00E94752289E30E9475228BE00E94752286E80E94752221968AEFC3
S1231A20C030D80709F45CC0D3CFC0E0D0E00E94C122823008F44CC00E945222892B09F0C6
S1231A4047C00E9452228C3A910509F049C083E50E94752288E00E9475228091B0059091DE
S1231A60B1050E9475228091B0059091B105892F99270E9475228091EA059091EB050E9472
S1231A8075228091EA059091EB05892F99270E9475228091E5059091E6050E947522809198
S1231AA0E5059091E605892F99270E94752280911806909119060E94752280911806909183
S1231AC01906892F99270E9475228CEA0E94752221964AEFC030D40719F0A9CF0E9475220E
S1231AE0A895DF91CF911F910F91FF90EF90DF90CF9008950F931F93CF93DF931092ED0550
S1231B001092EC050E94BE213C9A3D9A3F9A3E9A449A459A479A469A38984098399841987F
S1231B203A9842983B984398389839983A983B9854985C9855985D9854985598239A269AE9
S1231B40279A2B9A2E982F98259A249A5398529822985698219820980E94C921AAE5B1E057
S1231B600E94BE23802D80938A050E941D1C0E94681C0E94AC210E94EE050E9449042B9AD6
S1231B802E98A7E0B0E00E94BE23802D12BC11BC85FF9BC080910001909101019F7D909346
S1231BA00101809300010E9445030E9492030E94C1000E9486000E94FD0086E0AAE0B0E040
S1231BC0082E0E94CB2389E1ABE0B0E0082E0E94CB238EE1ACE0B0E0082E0E94CB23AEE011
S1231BE0B0E0082E0E94CB2320E030E0F901E05EFC4F8081D901A25ABE4F082E0E94CB234E
S1231C002F5F3F4F2A30310589F780912501A9E6B1E0082E0E94CB2380912601AAE6B1E01E
S1231C20082E0E94CB2380912701ABE6B1E0082E0E94CB2380912801ACE6B1E0082E0E9484
S1231C40CB2320E030E0F901EF53FA4F8081D901AE58BE4F082E0E94CB232F5F3F4F2A30D3
S1231C60310589F720E030E0F901EF53FA4F8089D901A458BE4F082E0E94CB232F5F3F4F47
S1231C802A30310589F78091E405A1E7B1E0082E0E94CB23809114019091150166E070E064
S1231CA00E945A23ADE0B0E0062E0E94CB2384E1ADE6B1E0082E0E94CB2381EEAEE6B1E03D
S1231CC0082E0E94CB2312BC11BC0E94E8000E9411010E949A000E946100809100019091EF
S1231CE0010185FD07C080916F008B7F80936F00449A459A80912401882311F480E801C0BD
S1231D0080E48093360110921B0580911401909115018D5D954030F08CED95E090931501EC
S1231D20809314011092790586B3866086BB78948AEA0E94752280E00E94752285E50E9499
S1231D40752289B1829586958695817080938B0580916E00836080936E002B9A2E9AA89520
S1231D6080917C0590917D058E37910570F180917905882351F58091EC059091ED059F7EBC
S1231D809093ED058093EC0580916F00856080936F0080916E00836080936E002B9A81E036
S1231DA0809379058091EC059091ED0580629093ED058093EC058091EC059091ED05906277
S1231DC09093ED058093EC0547C080917905813009F042C080917C0590917D058E37910514
S1231DE0D8F580916F008D7F80936F00809170008C7F8093700080916F008B7F80936F00E9
S1231E0080916E00836080936E008091EC059091ED058F7D9093ED058093EC058091EC059F
S1231E209091ED05877F9093ED058093EC05389839983A983B9854985598449A459A1092EE
S1231E4079058091EC059091ED059F7D9093ED058093EC0510927705809179058130F9F46B
S1231E60809177058823C1F080916F00826080936F008091700083608093700080916E002B
S1231E80836080936E008091EC059091ED0588609093ED058093EC052B9A2E9A13C01092C2
S1231EA07705449A459A109277051092B300109283051092820580913E0190913F01892BBA
S1231EC009F42B9840917C0550917D052091200130912101809100019091010180709074AB
S1231EE0822B932B4817590788F48091EC059091ED0597FD0BC08091EC059091ED059F7B95
S1231F009093ED058093EC05469A0AC08091EC059091ED0590649093ED058093EC054698FA
S1231F20F89480918405909185058A5A9A4AC1F080918405909185058555954589F07894D5
S1231F408091EC059091ED0580649093ED058093EC0588EE93E090933301809332010AC01B
S1231F6078948091EC059091ED058F7B9093ED058093EC05F89480918605909187058A5A60
S1231F809A4AC1F080918605909187058555954589F078948091EC059091ED058068909306
S1231FA0ED058093EC0588EE93E090933301809332010AC078948091EC059091ED058F77B0
S1231FC09093ED058093EC0580913201909133010B9758F02F9A8091320190913301019767
S1231FE0909333018093320101C02F9880911B05833009F4FBC0843018F4882371F08EC002
S1232000853009F433C2853008F45DC1863009F4EBC1873009F0E3C271C280917A059091AE
S12320207B058D52914008F4DDC2E0911B05F0E080917800909179008C7F65E070E00E940B
S12320405A236D5F7F4FEE0FFF1FE85AFA4F7183608380911B05C82FD0E0E0911B05F0E0AF
S1232060EE0FFF1FE45EFA4F80819181E0911B05F0E0EE0FFF1FE85AFA4F20813181880FB2
S1232080991F880F991F820F931F880F991F6AE070E00E945A23CC0FDD1FC45EDA4F7983CC
S12320A0688310927B0510927A0580911B058F5F80931B0580911B05806480937C000E9456
S12320C0E00780911C0590911D058035910564F42091140130911501C901880F991F820FB6
S12320E0931F9695879504C08091140190911501909317018093160180913E0190913F01AC
S1232100892B09F46AC280913E0190913F01019790933F0180933E012B9A5FC280917A056A
S123212090917B058D52914008F45CC290911B0540918E05842F83708450990F990F980F1A
S1232140E92FF0E0EE0FFF1FEE5FFE4F808191812091780030917900820F931F96958795DE
S12321609183808310927B0510927A05A89580911B05C42FD0E0813071F48E01085F1F4F76
S1232180842F0E94FA05000F111F045E1A4FF801918380830CC08081918162E070E00E94BA
S12321A06E23CC0FDD1FCC5CDA4F7983688380911B058F5F80931B0580911B058064809301
S12321C07C0080912C0590912D058D38910514F082E309C080912C0590912D058937910572
S12321E00CF400C289E180937805FCC180917A0590917B058D52914008F4F4C1E0911B053F
S1232200F0E080917800909179009695879596958795EE0FFF1FE85AFA4F9183808380916B
S12322201B05C82FD0E0E0911B05F0E0EE0FFF1FE45EFA4F80819181E0911B05F0E0EE0F5B
S1232240FF1FE85AFA4F20813181880F991F880F991F820F931F65E070E00E945A23CC0F0E
S1232260DD1FC45EDA4F7983688310927B0510927A0580911B058F5F80931B0580911B0566
S1232280806480937C000E94E007A89580918E058F5F80938E05843010F010928E0520912F
S12322A08E05922F91709295990F907E85B18F7D892B85B9220F220F220F207185B18F7E4D
S12322C0822B85B98FC180917A0590917B058159914008F487C180912401882331F1E0912B
S12322E01B05F0E08091780090917900969587959695879590E0EE0FFF1FE85AFA4F91830F
S12323008083A0911B05B0E0E0911B05F0E0EE0FFF1FE85AFA4F80819181AA0FBB1FA45E26
S1232320BA4F11969C938E933EC0E0911B05F0E08091780090917900EE0FFF1FE85AFA4F71
S12323409183808380911B05C82FD0E0E0911B05F0E0EE0FFF1FE45EFA4F00811181E091FF
S12323601B05F0E0EE0FFF1FE85AFA4F808191810E94BA069C01220F331F280F391FC801D6
S123238043E0880F991F4A95E1F7801B910B820F931F6AE070E00E945A23CC0FDD1FC45EE4
S12323A0DA4F7983688310927B0510927A0580911B058F5F80931B0580911B05806480934C
S12323C07C0020918B0589B1829586958695817030E090E02817390709F4FFC0E0918F0504
S12323E0F09190050995F9C080917A0590917B058D52914008F4F6C0E0911B05F0E0809167
S12324007800909179009695879596958795EE0FFF1FE85AFA4F9183808380911B05C82F33
S1232420D0E0E0911B05F0E0EE0FFF1FE45EFA4F80819181E0911B05F0E0EE0FFF1FE85A10
S1232440FA4F20813181880F991F880F991F820F931F880F991F6AE070E00E945A23CC0F18
S1232460DD1FC45EDA4F798368833EC080917A0590917B058D52914008F4B4C0E0911B054A
S1232480F0E080917800909179009695879596958795EE0FFF1FE85AFA4F91838083E09189
S12324A01B05F0E0EE0FFF1FE85AFA4F2081318184E190E0FC012E9FC0012F9F900D3E9F87
S12324C0900D11240E9460069093270580932605809126059091270562E070E00E946E2343
S12324E0709327056093260510927B0510927A0580911B058F5F80931B0568C080917A053E
S123250090917B058D52914008F46CC0E0911B05F0E0809178009091790096958795969548
S1232520879590E0EE0FFF1FE85AFA4F918380838091660590916705893791050CF1A091C1
S12325401B05B0E0E0911B05F0E0EE0FFF1FE45EFA4F40815181E0911B05F0E0EE0FFF1FB1
S1232560E85AFA4F20813181CA01880F991F840F951F820F931F969587959695879519C06E
S1232580A0911B05B0E0E0911B05F0E0EE0FFF1FE45EFA4F20813181E0911B05F0E0EE0F9E
S12325A0FF1FE85AFA4F80819181820F931F96958795AA0FBB1FA45EBA4F11969C938E933C
S12325C010927B0510927A0510921B0580911B05806480937C000E94E007A89503C081E064
S12325E080931B0580917A0590917B05019690937B0580937A0580917C0590917D058F558E
S1232600914008F442C0809110068F5F8093100690911006809111069817D0F11092100622
S123262080912A0590912B05E0911C06FF27E7FDF095E251FA4F208130E08217930734F45B
S123264080910E0690910F06890F17C080912A0590912B05E0911C06FF27E7FDF095E251C6
S1232660FA4F208130E0821793074CF080910E0682302CF080910E06815080930E068091CC
S12326800E0685362CF084E601C081E080930E0680917C0590917D058739910508F461C0F0
S12326A020912805309129058091220190E04996281739070CF055C08091B8059091B90589
S12326C001969093B9058093B8052091B8053091B9058091BA059091BB052817390708F495
S12326E042C01092B9051092B80520917C0530917D058091B2059091B3052817390730F45C
S12327009091B6058091B705890F15C020917C0530917D058091B2059091B3054996821711
S1232720930758F49091B6058091B505891728F48091B60581508093B6059091B6058091F4
S1232740B405891718F48091B40508C09091B6058091B505981738F48091B5058093B60563
S123276002C01092B60580911A0582FF1BC080917C0590917D05805D9740A0F4209128054F
S1232780309129058091220190E00596281739074CF481E080938D058091EC059091ED052D
S12327A0916007C010928D058091EC059091ED059E7F9093ED058093EC05809100019091AB
S12327C0010192FF27C020917C0530917D0580912C0190912D0182179307E0F420917C0540
S12327E030917D0580912E0190912F012817390788F420912805309129058091220190E095
S123280005962817390734F48091EC059091ED05946005C08091EC059091ED059B7F909352
S1232820ED058093EC05809100019091010193FF28C04A9926C020917C0530917D058091A0
S12328403001909131018217930730F48091EC059091ED05986005C08091EC059091ED05B2
S1232860977F9093ED058093EC0580911A0583FF29C080917C0590917D05875D9640C0F4E7
S123288021C0809100019091010193FF21C0199B1FC080911A0583FF15C08091940587352B
S12328A088F480912A0590912B058837910554F48091BC059091BD0588609093BD058093D5
S12328C0BC053FC08091BC059091BD05877FF5CF8091BC059091BD05877F9093BD05809302
S12328E0BC058091350120912A0530912B0590E082179307BCF040917C0550917D05209146
S12329001E0130911F01809100019091010180709078822B932B8417950750F480911A0570
S123292080FF06C08091EC059091ED05986005C08091EC059091ED05977F9093ED05809329
S1232940EC05809100019091010180FF67C080912B0180FF11C08091AF05883C28F0809168
S1232960B6058823B9F418C09091B6058091AF058695891790F010C080912B0182FF0DC031
S12329808091AF05883C48F08091EC059091ED0596FF02C0549A01C0549880912B0184FFAB
S12329A016C08091AF05883C28F080910E0618165CF12CC020910E068091AF05332727FD08
S12329C03095869590E0821793070CF11FC080912B0186FF1CC08091AF05883CC0F020910C
S12329E07C0530917D058091190190911A018217930760F420912A0530912B0580917605C4
S1232A0090E08217930714F4559A01C055988091AF05883C28F01092AF0502C054985598D8
S1232A208091AF058F5F8093AF0598C91F920F920FB60F9211248F939F9380911D068F5F54
S1232A4080931D0680911D06882309F446C08091EC059091ED0590619093ED058093EC053B
S1232A60109279058091EC059091ED059F7D9093ED058093EC0580916F008B7F80936F00DC
S1232A8080916F008D7F80936F00809170008C7F8093700080916E00836080936E00449A54
S1232AA0459A8091EC059091ED058F7D9093ED058093EC058091EC059091ED05877F9093BB
S1232AC0ED058093EC05389839983A983B985498559810927D0510927C0578949F918F913A
S1232AE00F900FBE0F901F9018951F920F920FB60F9211248F9380912A01813019F482E000
S1232B008093C0058F910F900FBE0F901F9018958091AA05882309F466C02091AA05809153
S1232B20AA05823089F4449A8091860590918705880F991F90938705809386058091860554
S1232B409091870581600BC08091AA05803269F4459A8091860590918705880F991F9093AF
S1232B608705809386051092AA0580918400909185009093B1058093B005479A8091E5051E
S1232B809091E605892B61F080911A06882341F08091E5059091E60590938B0080938A00C1
S1232BA080917C0590917D058C5D954008F04FC080911A0581FF4BC080918A0090918B0015
S1232BC088539F4F90938B0080938A0020931A0680918A0090918B008C509E4F90931906B8
S1232BE080931806089580911A06882381F120911A06223089F444988091840590918505F4
S1232C00880F991F9093850580938405809184059091850581600BC020911A06203269F4A7
S1232C2045988091840590918505880F991F90938505809384052093AA0580911806909124
S1232C40190690938B0080938A0010921A0608951F920F920FB60F9211242F933F934F9344
S1232C605F936F937F938F939F93AF93BF93EF93FF930E9488152B9A7894FF91EF91BF91DE
S1232C80AF919F918F917F916F915F914F913F912F910F900FBE0F901F9018951F920F9277
S1232CA00FB60F9211242F938F939F93F8942091130120959091C005943001F1953040F4C4
S1232CC0923019F19330A0F4913009F049C008C0973169F19336A9F19E3009F041C01BC01A
S1232CE02093B20084E08093B100389A83E042C026BD83E085BD3A9A84E03CC02093B200EB
S1232D009093B1003B9A82E035C026BD83E085BD399A81E02FC081E0809303052093B20023
S1232D2084E08093B100389A3B9A87E123C081E08093040526BD83E085BD399A3A9A8EE05B
S1232D4019C081E0809303052093B20084E08093B100389A3B9A3A9A399A9093C0050CC08B
S1232D602093B20084E08093B100389A3B9A3A9A399A83E68093C00578949F918F912F9117
S1232D800F900FBE0F901F901895CF93DF93EC0180918905E7E0F0E0E81BF109EE0FFF1FB9
S1232DA0E45EFA4F8081918120918805821B282F30E08091290190E0880F991F880F991FE6
S1232DC0AC01429FC001439F900D529F900D112464E670E00E945A236436710520F083E61C
S1232DE080931B0602C060931B0680911B066AE00E944E2380931406809114068A301CF018
S1232E0089E08093140680917C0590917D058D5E9340C0F580917C0590917D0564E670E0A1
S1232E200E945A236550609317068091170618161CF01092170607C08091170685301CF0CD
S1232E4085E080931706E0911706FF27E7FDF095E75CFE4F808190E09093BF058093BE05FE
S1232E60109212068FEF80931C0680911406992787FD909534E0880F991F3A95E1F7809330
S1232E808005C7C080917C0590917D05875F9242E8F086E9809312068FE080931C0680910C
S1232EA0140690911C068295807F890F80938005E0918005F0E0E05CFE4F808190E0880F14
S1232EC0991F9093BF058093BE05A3C080917C0590917D05885E934062E370E00E945A2374
S1232EE060931206809112066AE00E944E2380931C068091140690911C068295807F890FEC
S1232F0080938005E0918005F0E0E05CFE4F808190E0880F991F9093BF058093BE05809138
S1232F201C0687FD39C080911C068F30ACF5E0918005F0E0EF5BFE4F8081E0918005F0E037
S1232F40E05CFE4F6081E091BE05F091BF052091120640911C06861B880F992787FD90952D
S1232F6030E06AE04602A0011124241B350BAC01429FC001439F900D529F900D11246AE07B
S1232F8070E00E946E23772767FD70956E0F7F1F7093BF056093BE058091140687FD39C063
S1232FA0809114068930ACF5E0918005F0E0E05BFE4F8081E0918005F0E0E05CFE4F608109
S1232FC0E091BE05F091BF0520911B0640911406861B880F992787FD909530E06AE0460274
S1232FE0A0011124241B350BAC01429FC001439F900D529F900D11246AE070E00E946E231A
S1233000772767FD70956E0F7F1F7093BF056093BE0580917C0590917D05855F914010F41F
S12330205AEB69C080917C0590917D058952934210F05DE060C080917C0590917D058556CC
S12330409941B8F080917C0590917D05845699416AE070E00E945A23CB01880F991F880F96
S1233060991F860F971F64E670E00E945A23562F42C080917C0590917D05815A9F40B8F072
S123308080917C0590917D05805A9F406AE070E00E945A23CB01F3E0880F991FFA95E1F730
S12330A064E670E00E945A23562F545124C080917C0590917D05855F914010F450E01BC04C
S12330C080917C0590917D05845F91406AE070E00E945A23CB019B01E3E0220F331FEA951D
S12330E0E1F7880F991F820F931F64E670E00E945A23562F57532091BE053091BF05852FCD
S1233100992787FD9095820F931F97FF06C08091BE059091BF0551E0581B40919405445642
S123312045310CF044E12091BE053091BF05809112019091780520583040280F311D291B88
S12331403109842F4C3E0CF48CEE682F772767FD7095620F731F852F992787FD9095680F45
S1233160791F42E0693574072CF068E572E080E090E00CC0653071052CF465E070E080E001
S123318090E004C0882777FD8095982F20917E0530917F052C0F3D1F40E050E00E942F23A4
S12331A028E037E040E050E00E948123C21BD30BCE01DF91CF910895CF93DF93EC016091AD
S12331C0AC057091AD052091130126952695620F711D7695679580E090E02AE530E040E037
S12331E050E00E942F2320917E0530917F052C0F3D1FE3E036952795EA95E1F740E050E0A6
S12332000E948123E0911C06FF27E7FDF095E051FB4FE08164EB70E06E1B7109882777FDA1
S12332208095982F620F731F841F951F9E0140E050E00E942F2322E130E040E050E00E946C
S12332408123CA01B9012AE030E040E050E00E9481232A97CE01A0E0B0E02A9682179307FE
S1233260A407B50718F48AE090E003C0CE01821B930BDF91CF9108951F93CF93DF9380912C
S1233280840090918500909322068093210680918400909185008639910508F4A3C2809179
S12332A01D06882349F088EE9DEF909302058093010510921D065BC08091840090918500A3
S12332C060910105709102059B0136952795AB01E3E056954795EA95E1F7241B350B821723
S12332E0930768F481E08093200680912A01823009F078C28091EF048093C00573C28091F7
S12333007C0590917D05E0917E05F0917F0520918400309185008091EE0490E0261B370B1B
S1233320AC01429FC001439F900D529F900D11246EE170E00E946E23CB018E0F9F1F62E0BD
S123334070E00E946E2370937F0560937E0510927F0510927E058091840090918500909340
S1233360020580930105109285001092840080917705893628F4809177058F5F809377056A
S123338080917C0590917D058052934040F4449B02C0459904C0449A459A1092AA054798EB
S12333A080917C0590917D05C0910105D0910205D093EB05C093EA052091EA053091EB052F
S12333C01091810040E050E060E070E489E191E00E94A323CA01B9012EE130E040E050E0AC
S12333E00E942F2320EC129F9001112420503240442737FD4095542F0E94812330937D05EE
S123340020937C052091A1053091A20540919F055091A005C901880F991F820F931F840FCB
S1233420951F96958795969587959093A2058093A10580919D0590919E059093A005809371
S12334409F0580919B0590919C0590939E0580939D058091990590919A0590939C05809390
S12334609B05809197059091980590939A0580939905809195059091960590939805809390
S1233480970580917C0590917D05909396058093950580917C0590917D058D5D9540D8F030
S12334A04091940580919505909196052091A1053091A205821B930B23E0429FA001112483
S12334C0840F951F24E0969587952A95E1F78B5A809394050FC084E68093940580917E05B5
S12334E090917F0564E070E00E946E2370937F0560937E0510921D0680917C0590917D0565
S12335008C52914000F5809181008330E1F4809120068823C1F484E0809381001092850033
S123352010928400D695C795D695C795D0930205C09301058091EA059091EB0596958795B8
S12335409695879526C080917C0590917D058D5B924018F1809181008430F9F480912006D8
S12335608823D9F483E0809381001092850010928400CC0FDD1FCC0FDD1FD0930205C09320
S123358001058091EA059091EB05880F991F880F991F9093EB058093EA058091EA0590913C
S12335A0EB050E94C516909319068093180680917C0590917D058A58924018F488EE93E049
S12335C009C080917C0590917D058E57944038F488EC90E090931F0680931E0604C010923B
S12335E01F0610921E068091180690911906209116013091170140911E0650911F06821B34
S1233600930B841B950B9093160680931506809115069091160697FF20C080911506909130
S123362016062091EA053091EB054091180650911906820F931F8417950778F42091EA05A4
S12336403091EB058091180690911906821B930B44969093160680931506F89480917C05A6
S123366090917D05805E9E4208F091C08091EC059091ED0593FD8BC0809115069091160643
S12336808536910504F11092AA05809115069091160690938B0080938A0080918A0090911F
S12336A08B009093E6058093E50580912006882311F480E201C082E080931A061092AA0580
S12336C084E090E058C080911506909116068B5B9F4F2CF11092AA0584E690E090938B00C7
S12336E080938A009093E6058093E50580912006882329F480E280931A06459804C082E087
S123370080931A0644981092AA0588E290E09093E8058093E70584E18093000530C08091DE
S123372018069091190690938B0080938A002091EA053091EB058091150690911606820F91
S1233740931F9093E6058093E50580912006882331F4459880E28093AA0582E005C044989D
S123376082E08093AA0580E280931A0684E18093000584EB90E09093E8058093E70510927F
S123378020068091EC059091ED059F770FC08091EA059091EB058C509E4F90938B0080936A
S12337A08A008091EC059091ED0590689093ED058093EC0580917C0590917D058D5A9D405C
S12337C038F080918400909185008C599F4F06C08091EA059091EB050E94DC189093890096
S12337E0809388007894DF91CF911F9108951F920F920FB60F9211242F933F934F935F93AC
S12338006F937F938F939F93AF93BF93EF93FF930E943C192B9A7894FF91EF91BF91AF912C
S12338209F918F917F916F915F914F913F912F910F900FBE0F901F9018951092800081EFCB
S12338409FEF909389008093880085EF9FEF90938B0080938A0080E880938100109285001F
S12338601092840083E08093810080916F00876080936F00539852983C9A3D9A449A459AFF
S1233880A2E0B2E00E94BE23802D8093EE04A1E0B2E00E94BE23802D8093EF048091EF048E
S12338A08E3039F08091EF04873119F087E18093EF0480918A05813021F4809169008C601E
S12338C003C080916900886080936900E99A089521EB30E0F90110821092B6001092B200CF
S12338E01092B300A0E7B0E08C9183608C9338984098399841983A9842983B9843983898BD
S123390039983A983B98EFE6F0E080818D7F80838C918C7F8C9386E0F901808384E6809351
S1233920E1050895813099F438983B9880912A01843021F439983A981092040510922606FE
S123394010922506109203051092B1000895823049F439983A981092240610922306109231
S1233960040515BC08951F920F920FB60F9211242F933F934F935F936F937F938F939F930F
S1233980AF93BF93EF93FF93F89480910305843019F481E00E94921C7894FF91EF91BF91F8
S12339A0AF919F918F917F916F915F914F913F912F910F900FBE0F901F9018950F931F9348
S12339C080911C0590911D050A9714F487E003C080918D0586E08093B1001092B200809169
S12339E07C0590917D05845F914018F41092170616C080917C0590917D058D56974020F04B
S1233A008EE0809317060BC080917C0590917D0564E670E00E945A23655060931706E09115
S1233A201706F0E0E65DFC4F80818093130180918D05882329F02091F0018091180108C0E4
S1233A40E0918005F0E0E052FE4F808120911801829FC00111249093AD058093AC05809191
S1233A607C0590917D05825C914048F5809100019091010182FF19C08091AC059091AD050E
S1233A8020911B01820F911D9093AD058093AC058091EC059091ED0584609093ED0580935C
S1233AA0EC058EE18093AB053FC08091EC059091ED058B7F9093ED058093EC0535C08091A2
S1233AC0EC059091ED058B7F9093ED058093EC058091AB05823028F08091AB05815080938B
S1233AE0AB05E091AC05F091AD0580911B0120911B014091AB05E80FF11D8EE190E0841BBF
S1233B00910930E0AC01429FC001439F900D529F900D11246EE170E00E945A23E61BF70BA5
S1233B20F093AD05E093AC0580918D05882309F0ABC1E0918005F0E0E052FE4F808120917E
S1233B401801829FC00111249093AD058093AC0580911C0687FD3EC080911C068F30D4F528
S1233B60E0918005F0E0EF51FE4F6081E0918005F0E0E052FE4F40810091AC051091AD0572
S1233B808091120620911C06E091180170E0641B710990E04AE0240290011124821B930B91
S1233BA09C01629FC001639F900D729F900D11246AE070E00E946E23F0E06E9FC0016F9FA7
S1233BC0900D7E9F900D1124800F911F9093AD058093AC058091140687FD3EC080911406A5
S1233BE08930D4F5E0918005F0E0E051FE4F6081E0918005F0E0E052FE4F40810091AC05D2
S1233C001091AD0580911B0620911406E091180170E0641B710990E04AE0240290011124F7
S1233C20821B930BAC01649FC001659F900D749F900D11246AE070E00E946E23F0E06E9FA4
S1233C40C0016F9F900D7E9F900D1124800F911F9093AD058093AC058091000190910101F8
S1233C6084FF55C02091460530914705809128059091290528173907C4F48091280590917C
S1233C8029052091460530914705821B930B64E070E00E946E2380918105861710F46093BC
S1233CA08105809123018093AE053091AE053430C8F08091AC059091AD05E0918105F0E093
S1233CC0E05EFC4F2081820F911D9093AD058093AC0531503093AE058091EC059091ED05D2
S1233CE0806109C0109281051092AE058091EC059091ED058F7E9093ED058093EC0580914D
S1233D002805909129059093470580934605809100019091010191FFB4C080918B058823D1
S1233D2009F0AFC08091E3058F5F8093E3059091E3058091E405981708F4A6C01092E30597
S1233D408091240590912505E0911406FF27E7FDF095EF53FA4F208130E028173907B4F45D
S1233D608091240590912505E0911406FF27E7FDF095EF53FA4F2081821B910962E070E0AB
S1233D800E946E236C596093E1052BC08091240590912505E0911406FF27E7FDF095EF5382
S1233DA0FA4F208130E082179307DCF48091E1051816BCF4E0911406FF27E7FDF095EF53D1
S1233DC0FA4F8081209124053091250590E0821B930B62E070E00E946E2384E6861B809342
S1233DE0E1058091EC059091ED059D7F9093ED058093EC052091E105E0911406FF27E7FD63
S1233E00F095EF53FA4F8089332727FD309590E08C599F4F8217930754F4E0911406FF27D3
S1233E20E7FDF095EF53FA4F80898C591EC02091E105E0911406FF27E7FDF095EF53FA4F82
S1233E404089332727FD309584E690E0841B910928173907CCF4E0911406FF27E7FDF095E6
S1233E60EF53FA4F908984E6891B8093E1058091EC059091ED0592609093ED058093EC0573
S1233E8003C084E68093E105209132053091330580911D0190E0C29628173907D4F58091C7
S1233EA000019091010181FF34C08091320590913305C397D4F040911C0180911C012091DA
S1233EC032053091330560911D0190E070E06E5C7F4FFC01E29FC001E39F900DF29F900DBB
S1233EE011240E945A23461B03C080911C01482F50E08091AC059091AD05480F591F50932A
S1233F00AD054093AC058091EC059091ED05826005C08091EC059091ED058D7F9093ED0575
S1233F208093EC0580912401882371F02091AC053091AD058091E10524563040992787FD3D
S1233F409095280F391F0DC02091AC053091AD058091E1052C593F4F992787FD9095281B51
S1233F60390B3093AD052093AC058091BC059091BD0583FF1CC0E091AC05F091AD05209107
S1233F8038018091AC059091AD0564E170E00E946E2330E0629FC001639F900D729F900D68
S1233FA011248E0F9F1F9093AD058093AC05809100019091010190FF4CC080911C059091B1
S1233FC01D05823891050CF044C08091AC059091AD0520912501820F911D9093AD058093D8
S1233FE0AC05E0911C05F0911D05609118012091250182E890E08E1B9F0B70E0AB01849FAA
S1234000B001859F700D949F700D11248FEF90E0FB01E89FB001E99F700DF89F700D1124F5
S1234020882777FD8095982F30E040E050E00E942F2320E43FE140E050E00E94812380915E
S1234040AC059091AD05820F931F9093AD058093AC052091AC053091AD058091180145EFC9
S1234060849FC00111248217930754F480911801849FC00111249093AD058093AC050BC001
S12340808091AC059091AD051816190624F01092AD051092AC0520918205309183058091ED
S12340A0AC059091AD05820F931F96958795909383058093820540917C0550917D05209143
S12340C01E0130911F01809100019091010180709078822B932B4817590730F48091EC055F
S12340E09091ED059F770DC080911A0580FD04C0389839983A983B988091EC059091ED05FA
S123410090689093ED058093EC058091EC059091ED0592FF04C0389839983A983B987894CE
S12341201F910F9108951F920F920FB60F9211242F933F934F935F936F937F938F939F93D1
S1234140AF93BF93EF93FF93F89480910305823039F1843039F1813051F50E94DE1C8091B0
S1234160820590918305909326068093250680912506909126068F3F910561F058F08091E7
S12341802506909126068F5F8093B30082E0809303050DC080912506909126068093B30056
S12341A084E0F5CF81E00E94921C109203057894FF91EF91BF91AF919F918F917F916F916C
S12341C05F914F913F912F910F900FBE0F901F9018951F920F920FB60F9211242F933F9393
S12341E04F935F936F937F938F939F93AF93BF93EF93FF93F89480912A018430A8F58091AD
S12342000405823031F0843059F1813009F05AC002C084E01AC08091820590918305909398
S123422024068093230624E025BD16BC80912306909124068F3F910559F050F080912306B0
S1234240909124068F5F87BD82E0809304053AC0809123069091240687BD2093040532C0EE
S123426082E00E94921C2EC080912B0181FD04C080912B0185FF23C084E085BDE0918005DB
S1234280F0E0E058FD4F80818C5E87BD8091EC059091ED0597FD16C08091EC059091ED0503
S12342A092FD10C087B58F3168F080912B0181FD549A80912B0185FF05C0559A03C016BC94
S12342C081E087BD7894FF91EF91BF91AF919F918F917F916F915F914F913F912F910F902A
S12342E00FBE0F901F9018951F920F920FB60F9211242F933F934F935F936F937F938F9367
S12343009F93AF93BF93EF93FF93F89480912A01843040F480910405843061F482E00E94E8
S1234320921C08C080912B0181FD549880912B0185FD55987894FF91EF91BF91AF919F91D4
S12343408F917F916F915F914F913F912F910F900FBE0F901F90189554985C9855985D98A0
S12343605498559815BCEEE6F0E080818360808384E085BD16BC82E187BD089511B88FEF01
S123438084B915B887B98AB90895089508950895089588E98093C10083E18093C4008EE687
S12343A096E090932C0680932B0690932806809327068EE296E090932A06809329069093BB
S12343C0AF068093AE0610922D061092E90508951F920F920FB60F9211248F939F93EF9398
S12343E0FF9380912D06882311F1E0912B06F0912C0681918093C600F0932C06E0932B069D
S1234400EE5AF64030F08EE696E090932C0680932B0680912D06815080932D0680912D06D8
S1234420882329F48091C1008F7D8093C100FF91EF919F918F910F900FBE0F901F90189537
S12344401F920F920FB60F9211242F938F939F93EF93FF938091C600E091AE06F091AF060F
S123446080838091E9058F5F8093E9058091AE069091AF0601969093AF068093AE068E5692
S1234480964030F08EE296E09093AF068093AE06FF91EF919F918F912F910F900FBE0F9072
S12344A01F9018958091E905882319F48FEF9FEF0895F8948091E90581508093E905E0916E
S12344C02906F0912A062191F0932A06E0932906EE56F64030F08EE296E090932A0680930B
S12344E029067894822F90E00895982F80912D068F33E0F780912D06803418F080E090E04B
S12345000895F89480912D068F5F80932D06E0912706F09128069083809127069091280609
S1234520019690932806809327068E5A964030F08EE696E090932806809327068091C10024
S123454080628093C100789481E090E00895CF93DF93EC0104C00E94752281112196888117
S12345608823C9F781E090E0DF91CF91089585E095E00E94A72208958DE095E00E94A7225F
S123458008958091E90590E00895CF92DF92EF92FF920F931F93CF93DF93CDB7DEB7299789
S12345A00FB6F894DEBF0FBECDBF8C01F62EE42EDE011196E0E1F5E089E001900D92815067
S12345C0E1F749E06E010894C11CD11CFF2081F089E090E0841B91092F2D30E082179307C0
S12345E038F04150F601E40FF11D8CE28083FF244150F601E40FF11DC8016AE070E00E94E4
S12346005A23805D8083C8016AE070E00E945A238B01672B11F4FF2019F085E08F15B0F6BD
S123462019E01E197E010894E11CF11C07C0F701E10FF11D80810E9475221F5F1930B8F3B8
S123464029960FB6F894DEBF0FBECDBFDF91CF911F910F91FF90EF90DF90CF900895629FB6
S1234660D001739FF001829FE00DF11D649FE00DF11D929FF00D839FF00D749FF00D659FE7
S1234680F00D9927729FB00DE11DF91F639FB00DE11DF91FBD01CF0111240895991B79E033
S12346A004C0991F961708F0961B881F7A95C9F780950895AA1BBB1B51E107C0AA1FBB1FC5
S12346C0A617B70710F0A61BB70B881F991F5A95A9F780959095BC01CD01089597FB092EBF
S12346E007260AD077FD04D0E5DF06D000201AF4709561957F4F0895F6F7909581959F4F23
S12347000895A1E21A2EAA1BBB1BFD010DC0AA1FBB1FEE1FFF1FA217B307E407F50720F08F
S1234720A21BB30BE40BF50B661F771F881F991F1A9469F760957095809590959B01AC0106
S1234740BD01CF01089597FB092E05260ED057FD04D0D7DF0AD0001C38F4509540953095D9
S123476021953F4F4F4F5F4F0895F6F790958095709561957F4F8F4F9F4F0895F999FECF50
S1234780B2BDA1BDF89A119600B40895F7DFE02DF5DFF02D0895F999FECFB2BDA1BD00BC65
S12347A011960FB6F894FA9AF99A0FBE0895F3DF012CF1DF11240895FFCF2F0001000200CB
S12347C00300040005000600070008003228E803900106C409141E3C401F6419121E01018F
S12347E00203040A0411C4098813AC0D6400DCE64003020A14324696500054819596B7AF1F
S1234800C3C8BEBEB9B0AFAFADAC4984C0CBD2D6D7D0C7C2BBB8B3AEAAA9458AA2A9AAB79B
S1234820C0BABEBBB6B8B2B3B4B93281868DA4A58B8C8F9EA6A2A6A5A6C034525D5B596FEF
S1234840788285858281FF859FB034444E4B4A54615769727272737D9095272C1B252B334E
S12348604B5155616A6D6C7D828B1D211A242A32454C4F5E6169717E818634323232323211
S123488032323232327F3232323232323232323232323232323232323232131718191B1C21
S12348A01D1F21232527282C2E311418191A1C2124272B3035393C3E414316191D232A31FD
S12348C0353B3F42484E565A5E651B1D363E525863666C6E777D84898D932226434B617217
S12348E0818A9097A8ACAFB1B6B9292E484E6B7C939BA2AFB9BFCBD2D2D229344B536E7F6B
S12349009CA8B1BCC5D0D2D2D2D2283F4E587187A4B2BAC2D2D2D2D2D2D23746545E76910C
S1234920B1BEC4D2D2D2D2D2D2D239485660869FBAD2D2D2D2D2D2D2D2D20000000000000A
S1234940000000000000000000000000000000000000000000000000000000000000000053
S123496000000000000000000000000000000000000000000000000000000102030405061E
S12349800708090A0B0C0D0E0F100102030405060708090A0B0C0D0E0F1001020304050603
S12349A00708090A0B0C0D0E0F1014161718191A1B1C1D1E1F2021222324191A1B1C1D1E14
S12349C01F2021222324252627271E1F2022232425262728292A2B2C2D2E000204060708F1
S12349E0090A0C0E28262422201E1E1E1E1E1E1E1E1E1E1EF0FF80BBE0880465484BA4381E
S1234A00022BF0207019CC13860F440CC209D0074C061B052A046A03D1025602F201A10199
S1234A205F012801FB00D600B7009D0087007500660059004D0044003C0034002E002900B1
S1234A402500F0FF80BBE0880465484BA438022BF0207019CC13860F440CC209D0074C0645
S1234A601B052A046A03D1025602F201A1015F012801FB00D600B7009D00870075006600A7
S1234A8059004D0044003C0034002E0029002500F0FF80BBE0880465484BA438022BF02095
S1234AA07019CC13860F440CC209D0074C061B052A046A03D1025602F201A1015F012801AD
S1234AC0FB00D600B7009D0087007500660059004D0044003C0034002E0029002500F0FF86
S1234AE080BBE0880465484BA438022BF0207019CC13860F440CC209D0074C061B052A046B
S1234B006A03D1025602F201A1015F012801FB00D600B7009D0087007500660059004D00AE
S1234B2044003C0034002E00290025000000F5047E05AE066C08C00AB30D630F8B10D7111E
S1234B408813000000000A000F001E003C007800FA007201E00180028002000008000A0067
S1234B600C000E00C80A4A067E0484031A002000270032003E0066008E00B202EB0224035F
S1234B8037034B03560361037003E800D600C200B0009D008A00780078006500520040001B
S1234BA02D0019000700000001175A5A5A505050505050505050505050503200FA04041B1F
S1174BC05B481B5B324A000D0A002020202020202020200011
S503025F9B
